:020000040000FA
:100000008B0183160313FF3085008F309F00F03083
:10001000860081308100831241309F00860181017A
:100020000B110614A7200610A7200615061186142A
:100030008610F630A5002830A6005C30A7000730F7
:10004000A800B3012B20B3012B200608C039A9005A
:100050005F202B20282803102830AD002508A000A1
:100060002608A1002708A2002808A3000130A40048
:100070009D202C08B0002B08B100AF01B201AF20C9
:10008000061E4A280330B100A430B0003B30AF0058
:10009000B201AF2021083302031908002108B30080
:1000A0008611A40CA30CA20CA10CA00C031886159D
:1000B00006150611AD0B5028861486100800060898
:1000C000C039AA00AE000310AE0CAE0C2908AE0772
:1000D0000310AE0CAE0CAE0CAE0C2E0882078C28B2
:1000E0008F287F288E287F288C288E288F288F287D
:1000F0008E288C287F288E287F288F288C280130F6
:100100000B1D0A3081010B11A607031C8C2801303E
:10011000A707031C8C28A8072A08A900080001309B
:100120000B1D0A3081010B11A60203188C28013027
:10013000A70203188C28A8028C281F151F199E28B7
:100140001E08AB0083161E088312AC000800FF30A7
:10015000AE00000000000000AE0BA92808002F0828
:10016000A00730080318300FA10731080318310F1A
:0C017000A20732080318320FA307080092
:02400E00613F10
:00000001FF
